:020000001B28BB
:10000800FF00030E8301A7000A08A8008A01A20ABC
:100018000319A30A64003C308F00B0308E000C1026
:0E00280028088A00270E8300FF0E7F0E0900B5
:1000360083169F018F3081008312850183169901F3
:1000460007308312990007309A00F830831685002E
:100056006400113083129000C0308B003C308F005A
:10006600B0308E000C10013083168C008312A20172
:10007600A301A4010130A5000130A600051064000B
:100086008510051A6D28851A6D2800302302031D78
:100096004E28013022020318512805152308003C7A
:1000A600031D57282208013C031862282308003C38
:1000B600031D5F2822080F3C031C62280511230834
:1000C600003C031D682822080F3C03186C28A20177
:1000D600A3017D282E30FC007330FD00FD0B712836
:1000E600FC0B7128051A7A28851A7A287D28A5011D
:1000F600051405152508031D42280630FB0013309C
:10010600FC00AD30FD00FD0B8628FC0B8628FB0BA2
:100116008628000000000130A50064008519982893
:10012600051005118514A501A601051EA22824089F
:10013600003A031DA2280130A400A201A301051E56
:10014600B3282308003C031DAA282208233C0318D1
:10015600B328A5010510051185106400051AB028FD
:10016600051ABE282308003C031DBB282208233C91
:10017600031CBE28A4012508031D90280130A500F4
:100186002608031D42286400051185140230FB0071
:100196000430FC00BA30FD00FD0BCF28FC0BCF2845
:1001A600FB0BCF280000051185100230FB00043040
:1001B600FC00BA30FD00FD0BDE28FC0BDE28FB0B35
:0801C600DE280000C628E6282F
:02400E00C400EC
:00000001FF
